:020000040800F2
:1000000000200020B9000008CD0B0008E10B00081B
:1000100000000000000000000000000000000000E0
:10002000000000000000000000000000CD0B0008F0
:100030000000000000000000CD0B0008CD0B000800
:10004000CD0B0008CD0B0008CD0B0008CD0B000830
:10005000CD0B0008CD0B0008CD0B0008CD0B000820
:1000600000000000CD0B0008CD0B0008CD0B0008F0
:10007000CD0B0008CD0B000800000000E1000008D7
:1000800000000000CD0B0008000000000000000090
:100090006101000800000000CD0B0008CD0B000836
:1000A000CD0B0008CD0B0008CD0B0008590E000841
:1000B00035150008CD0B000800F004FD00F0C6FC6B
:1000C000E1235B02180000F01FFE62B6C04600F09C
:1000D00089FB024B180000F087FFFEE7508E0008F6
:1000E00080B500AF8023DB051A698023DB05012181
:1000F0008A431A61164B1B685A1C154B1A60144B25
:100100001B68180003F0E0F8021C124B1B68191C56
:10011000101C02F0C1FD031E00D116E00E4B1B683F
:10012000012B12D10D4B1B68002B0ED18023DB0558
:100130005B6B10331A008023DB05FF210A405A63F2
:10014000034B00221A6001F0A7FFC046BD4680BDE8
:10015000E801002000000020F0010020F401002050
:1001600080B500AF0B4B1A690A4B01218A431A6113
:10017000094B1B685A1C084B1A60074B1B68FA2B6B
:1001800004DD054B00221A6001F086FCC046BD4626
:1001900080BDC04600080140EC01002080B500AFE2
:1001A0003D4BDA6A3C4B01210A43DA62A023DB05AE
:1001B0001B68032293431A00A023DB0501210A4395
:1001C0001A60A023DB055A68A023DB0501218A43BE
:1001D0005A60A023DB051B680C2293431A00A0235E
:1001E000DB0504210A431A60A023DB055A68A0231B
:1001F000DB0502218A435A60A023DB051B683022FD
:1002000093431A00A023DB0510210A431A60A023A0
:10021000DB055A68A023DB0504218A435A60A0232A
:10022000DB051B68C02293431A00A023DB05402195
:100230000A431A60A023DB055A68A023DB050821C6
:100240008A435A60A023DB051B68144A1A40A02386
:10025000DB05802149000A431A60A023DB055A68A8
:10026000A023DB0510218A435A60A023DB051B680D
:100270000B4A1A40A023DB058021C9000A431A60FB
:10028000A023DB055A68A023DB0520218A435A609E
:10029000C046BD4680BDC04600100240FFFCFFFFC7
:1002A000FFF3FFFF80B500AF104BDA6A0F4B01215F
:1002B0000A43DA62A023DB051A68A023DB050C4998
:1002C0000A401A60A023DB05DA68A023DB05802141
:1002D00049040A43DA60A023DB05DA68A023DB05C2
:1002E00004490A40DA60C046BD4680BD00100240A5
:1002F000FFFFFFFCFFFFFFFD80B500AF0D4BDA6A8B
:100300000C4B02210A43DA620B4B1A680A4B032199
:100310000A431A60074BDA6A064B02210A43DA6283
:10032000054B1A68044B0C210A431A60C046BD46AF
:1003300080BDC046001002400004005080B500AFF0
:10034000A023DB05012252429A601B4BDA6A1A4B4A
:1003500001210A43DA62A023DB051B68174A1A4011
:10036000A023DB058021C9040A431A60A023DB0512
:100370005A69A023DB05802189010A435A61A02321
:10038000DB051A68A023DB050D490A401A60A0238B
:10039000DB05DA68A023DB058021C9030A43DA60A4
:1003A000A023DB05DA68A023DB0506490A40DA60F2
:1003B000C046BD4680BDC04600100240FFFFFFF3AF
:1003C000FFFF3FFFFFFF7FFF80B500AF094BDA6AF9
:1003D000084B01210A43DA62A023DB051B68064AA9
:1003E0001A40A023DB05802149020A431A60C04657
:1003F000BD4680BD00100240FFFFFCFF80B500AF8E
:10040000A023DB051B68134A1A40A023DB058021CB
:1004100049010A431A60A023DB055A68A023DB05C3
:1004200040218A435A60A023DB051B680A4A1A4010
:10043000A023DB058021C9010A431A60A023DB0544
:100440005A68A023DB0580218A435A60C046BD4616
:1004500080BDC046FFCFFFFFFF3FFFFF80B500AF6D
:10046000294BDA6A284B02210A43DA62274B1A68C1
:10047000264B27490A401A60244BDA68234B802117
:10048000C9010A43DA60214BDA68204B21490A404E
:10049000DA601E4B1A681D4B1F490A401A601B4B3D
:1004A000DA681A4B802149010A43DA60174BDA688F
:1004B000164B1A490A40DA60144B1A68134B184954
:1004C0000A401A60114BDA68104B8021C9000A43B8
:1004D000DA600E4BDA680D4B12490A40DA600B4BBA
:1004E0001A680A4BC0218A431A60084BDA68074B26
:1004F00040210A43DA60054BDA68044B80218A43C5
:10050000DA60C046BD4680BD0010024000040050C5
:10051000FF3FFFFFFF7FFFFFFFCFFFFFFFDFFFFF7B
:10052000FFF3FFFFFFF7FFFF80B582B000AF7860F9
:10053000A023DB051B697A6813405A425341DBB2A2
:100540001800BD4602B080BD80B582B000AF7860B3
:10055000054B1B697A6813405A425341DBB21800BD
:10056000BD4602B080BDC0460004005080B582B0D8
:1005700000AF786039603B687A680749074805F042
:100580008FFE064B01220221180001F079FCC046C3
:10059000BD4602B080BDC046EC8D0008D8010020E9
:1005A00090B587B002AFF860B9607A603B60F868D8
:1005B00004F07AFC02000B00174C1848B96800914F
:1005C000210005F06DFE154A154B1100180005F0CD
:1005D000A3FD124B01220121180001F051FC7868A3
:1005E00004F062FC02000B000E4C0C4839680091CC
:1005F000210005F055FE094A094B1100180005F0CD
:100600008BFD064B01220221180001F039FCC04687
:10061000BD4605B090BDC046F88D0008D801002049
:10062000048E00080C8E000880B582B000AF7860A0
:10063000786804F039FC0022094B03F0CFF902007E
:100640000B000849084805F02BFE074B0122012149
:10065000180001F015FCC046BD4602B080BDC04682
:1006600000408F40188E0008D801002080B582B06D
:1006700000AF00237B608020FFF766FF031E21D0C0
:100680001E2000F0ADFD8020FFF75EFF031E19D095
:100690000E4B1B685A1C0D4B1A600C4B1B68032B2E
:1006A00006D10A4B00221A6002E07B6801337B60AE
:1006B0008020FFF749FF031E04D07A68FA235B000D
:1006C0009A42F2DBC046BD4602B080BD1002002057
:1006D00080B582B000AF00237B604020FFF734FF7D
:1006E000031E23D01E2000F07BFD4020FFF72CFFCF
:1006F000031E1BD00F4B1B685A1C0E4B1A600D4B70
:100700001B68032B02D10B4B00221A6000237B6075
:1007100002E07B6801337B604020FFF715FF031E7A
:1007200004D07A68FA235B009A42F2DBC046BD46E9
:1007300002B080BD1402002080B500AF2020FFF77A
:1007400003FF031E0FD01E2000F04AFD2020FFF7FC
:10075000FBFE031E07D0054B1B685A425341DBB218
:100760001A00024B1A60C046BD4680BDF40100204D
:1007700080B500AF0820FFF7E7FE031E26D01E203D
:1007800000F02EFD0820FFF7DFFE031E1ED08020A4
:10079000FFF7DAFE031E19D00E4B00221A600E4B33
:1007A000180005F045FD0D4B01220121180001F054
:1007B00067FB0B4B01220221180001F061FBFA23B9
:1007C0009B00180000F00CFD01F05CFEC046BD4629
:1007D00080BDC046F0010020248E0008308E000845
:1007E000388E0008B0B582B000AF00237B600023D4
:1007F0003B60FFF7A3FD96239B01180000F0F4FD7A
:1008000001F068F9FFF7CAFC01F015FBFFF74AFD9C
:10081000FFF772FDFFF7D8FDFFF720FEFFF7EEFDB3
:1008200001F002FC01F050F801F068FBFA235B00D4
:10083000180000F0D5FC744B180005F06DFC01F0B9
:1008400021FEFFF795FF80235B00180001F0A0FB5D
:100850000300180004F0F8FA00226C4B03F02CFFA0
:1008600002000B001000190004F066FB021C80233C
:100870001B065A40664B1A6080239B00180001F04B
:1008800087FB0300180004F0DFFA0022614B03F03D
:1008900013FF02000B001000190004F04DFB021CB6
:1008A00080231B065A405C4B1A605C4B00221A6086
:1008B00080235B011800FFF737FE031E1FD01E20A8
:1008C00000F08EFC80235B011800FFF72DFE031E55
:1008D00003D0524BFE2292051A6000233B6002E0D7
:1008E0003B6801333B6080235B011800FFF71CFE6F
:1008F000031E04D03A68FA235B009A42F0DBFFF74C
:10090000B5FEFFF7E5FE424B1A68454B1B68190020
:10091000101C01F0A5FE0200424B1A603E4B1A6803
:10092000414B1B681900101C01F026FE02003F4BD2
:100930001A603C4B1C683D4B1D68384B1B68181CEB
:1009400002F0A2FC03001A002900200001F0FEF8CA
:1009500001F0AEF8364B1B68181C01F00FF90300CC
:10096000180002F0B1FC021C314B1A60304B1B68BE
:10097000181C04F099FA02000B002E49080005F03B
:10098000CBFB2B4B1B682C49181C02F067F9031E8C
:100990001BD0274B1B682949181C02F07DF9031E48
:1009A00013D07B685A1C7A60002B13DB244B012286
:1009B0001A601F4B1A68234B1B68191C101C01F08E
:1009C00079FB021C1F4B1A6004E000237B601C4B68
:1009D00000221A60FFF7B0FE154B1B68181CFFF7CA
:1009E00023FE104B1A68114B1B6819001000FFF70B
:1009F000BDFD154B1B689B68180004F0A5FCC820C2
:100A000000F0EEFB1DE7C0463C8E000800B0A040A1
:100A1000FC01002000F09F400002002004020020A2
:100A20001002002008020020140200200C02002006
:100A3000F8010020488E00080080EC430000C84305
:100A4000F0010020000000200800002080B582B0E6
:100A500000AF164B7B60164B3B6007E07A68131DB6
:100A60007B603B68191D396012681A603A68114B47
:100A70009A42F3D304E03B681A1D3A6000221A60E0
:100A80003A680D4B9A42F6D30C4B3B6004E03B684E
:100A90001A1D3A601B6898473A68094B9A42F6D388
:100AA000C046C046BD4602B080BDC0469C95000809
:100AB00000000020D80100205C0400209C95000864
:100AC0009C95000880B500AF3B4B1A683A4B01215A
:100AD0000A431A60C046384B1B6804221340FAD000
:100AE000354B0122DA60C046334BDB680C221340E1
:100AF000042BF9D1314B1A68304B02210A431A609A
:100B00002E4B1A682D4B01210A431A602A4B9A6B0F
:100B1000294B802149050A439A63294B80221201FF
:100B20001A60C046264B5B6810221340FAD1224B54
:100B3000DA68214B23490A40DA601F4BDA681E4B02
:100B40008821C9030A43DA601B4A1B4BD268DA606A
:100B5000194A194BD268DA60174A174BD268DA6023
:100B6000154B1A68144B18490A401A60124B1A6840
:100B7000114B802149040A431A60C0460E4B1A6883
:100B800080239B041340F9D00B4BDA680A4B0321F6
:100B90008A43DA60084BDA68074B03210A43DA60BC
:100BA000C046054BDB680C2213400C2BF9D1C04624
:100BB000C046BD4680BDC046001002400020024035
:100BC00000700040FFFF02FFFFFFFFFE80B500AF97
:100BD000024B180000F008FAFEE7C046788E0008C5
:100BE00080B500AF024B180000F0FEF9FEE7C046EA
:100BF000A88E000890B585B000AF78603960184BBA
:100C00001B68002B02D101235B4224E00023FB6020
:100C10000AE0FB685A1CFA603A68D418114B1800B5
:100C200000F0ADF9030023707B68013B1A00FB68FC
:100C3000934205D20B4B180000F0CCF9031EE8D10B
:100C4000FB68002B06D03A68FB68D31800221A70A4
:100C5000FB6800E000231800BD4605B090BDC0460B
:100C6000B00200201802002080B584B000AF786088
:100C70003960224B1B68002B02D101235B4238E014
:100C80007B683F2B0BDCC0461D4B180000F0A2F91F
:100C900003004022D21A7B689A42F5D302E0022375
:100CA0005B4226E00023FB600BE03A68FB68D31848
:100CB0001A78134B1100180000F030F9FB6801336B
:100CC000FB607B68FA689A42EFD30E4B1B680822E0
:100CD00013400DD10B4B1A680A4B08210A431A60C6
:100CE000074B180000F04BF903001A00054B9A62FD
:100CF00000231800BD4604B080BDC046B0020020ED
:100D0000640200200038014080B584B000AF7860F4
:100D100072B6C046454B00229A64444B9A6C434BD2
:100D20005A64424B5A6C414B1A64414B00229A64FC
:100D30003F4B9A6C3E4B5A643D4B5A6C3C4B1A6489
:100D40003C4B01221A603C4B00221A603B4BDA6A92
:100D50003A4B01210A43DA62394BFB607968F86843
:100D600001F040FE0300FB60A023DB059A68A0238E
:100D7000DB058021C9020A439A60A023DB055A687B
:100D8000A023DB052F490A405A60A023DB051B681E
:100D90002D4A1A40A023DB05802109030A431A606B
:100DA000A023DB055A6AA023DB0540210A435A62CF
:100DB000A023DB051B68254A1A40A023DB05802100
:100DC00089030A431A60A023DB055A6AA023DB05C6
:100DD0008021C9000A435A62184B5A6B174B802175
:100DE000C9010A435A631A4B1A68194B6C210A430A
:100DF0001A60174B00225A60154B00229A60144B60
:100E0000FA68DA60124B1A68114B01210A431A6022
:100E1000104B1A680F4B802109050A431A6062B60D
:100E2000C046C046BD4604B080BDC0461802002082
:100E300064020020B0020020B40200200010024032
:100E40000048E801FFFDFFFFFFFFF3FFFFFFCFFFBB
:100E50000038014000E100E080B500AF084BDB69DD
:100E60008022134001D000F025F8054BDB692022D9
:100E7000134001D000F006F8C046BD4680BDC04614
:100E80000038014080B500AF074B5B6ADAB2074B10
:100E90001100180000F042F8031E02D0044B01229A
:100EA0001A60C046BD4680BD0038014018020020CF
:100EB000B402002080B500AF164B180000F08AF88D
:100EC000031E08D0134B180000F059F803001A0055
:100ED000114B9A621BE0104B1A680F4B08218A4392
:100EE0001A600D4BDB694022134005D00A4B1A6A89
:100EF000094B40210A431A62074BDB6980221340E9
:100F000005D0054B9A69044B10210A439A61C046EB
:100F1000BD4680BD640200200038014080B582B02B
:100F200000AF78600A00FB1C1A707B681A6C7B6843
:100F30005B6C9A4205D17B689B6C002B01D001232E
:100F400019E072B6C0467B681B6C591C7A68116444
:100F50007A68F91C0978D1547B689B6C5A1C7B68B1
:100F60009A647B681B6C402B02D17B6800221A6458
:100F700062B6C04600231800BD4602B080BD80B5F1
:100F800084B000AF78607B689B6C002B01D100239C
:100F90001CE072B6C0467B685B6C591C7A68516471
:100FA0000F22BA187968CB5C13707B685B6C402B9E
:100FB00002D17B6800225A647B689B6C5A1E7B6856
:100FC0009A6462B6C0460F23FB181B781800BD4612
:100FD00004B080BD80B582B000AF78607B689B6C48
:100FE0001800BD4602B080BD80B582B000AF786009
:100FF0000B4B1B68002B09D101235B420BE07B6884
:101000005A1C7A6019000120FFF72EFE7B681B78BE
:10101000002BF4D100231800BD4602B080BDC046AD
:10102000B002002080B582B000AF0200FB1D1A7034
:10103000FB1D19000120FFF717FEC046BD4602B098
:1010400080BD80B500AF044B1800FFF798FF030088
:101050001800BD4680BDC04618020020B0B584B05F
:1010600000AF786039601E4B1B68002B02D1012352
:101070005B4231E00023FB600B23FB1800221A7057
:1010800017E0C046174B1800FFF7A4FF031EF9D066
:101090000B257C19134B1800FFF771FF0300237019
:1010A000FB685A1CFA601A007B689B187A19127840
:1010B0001A703B68013BFA689A4204DA0B23FB186A
:1010C0001B780D2BDDD1FB68002B04DDFB687A68F3
:1010D000D31800221A70FB681800BD4604B0B0BDDA
:1010E000B00200201802002090B583B000AFFC1DB4
:1010F000FFF7A7FF03002370FB1D1B781800FFF705
:1011000091FFFB1D1B781800BD4603B090BDB0B524
:1011100084B000AF78603960214B1B68002B02D18E
:1011200001235B4237E00023FB600B23FB18002206
:101130001A701DE0C0461B4B1800FFF74BFF031E43
:10114000F9D00B257C19174B1800FFF718FF030087
:1011500023702C003B191B781800FFF763FFFB6816
:101160005A1CFA601A007B689B183A1912781A7098
:101170003B68013BFA689A4204DA0B23FB181B78A0
:101180000D2BD7D1FB68002B04DDFB687A68D318E0
:1011900000221A70FB681800BD4604B0B0BDC046FE
:1011A000B00200201802002080B500AF0A4B0B4AA5
:1011B0005A60094B00229A60074B05221A60C0460C
:1011C000054B1A6880235B021340F9D0024B0022C2
:1011D0001A60C046BD4680BD10E000E0FF7C000004
:1011E00080B584B000AF78600023FB6004E0FFF7B7
:1011F000DBFFFB680133FB60FA687B689A42F6D339
:10120000C046C046BD4604B080BD80B582B000AFC8
:101210000200FB1D1A70FB1D1B7819000F4801F01E
:10122000E1FB030019000E4801F0DCFB03005A1E2D
:101230000C4B5A600B4B00229A600A4B05221A6035
:10124000C046084B1A6880235B021340F9D0054B57
:1012500000221A60C046BD4602B080BD40420F0069
:101260000048E80110E000E080B584B000AF78608D
:101270000023FB6015E00B23FB1800221A7008E026
:10128000FA20FFF7C2FF0B217B181A787B18013276
:101290001A700B23FB181B78032BF1D9FB68013361
:1012A000FB60FA687B689A42E5D3C046C046BD46FB
:1012B00004B080BD80B582B000AF7860C0467B6866
:1012C0005A1E7A60002BFAD1C046C046BD4602B015
:1012D00080BDC04690B585B000AF78603960184BCE
:1012E0001B68002B02D101235B4224E00023FB603A
:1012F0000AE0FB685A1CFA603A68D418114B1800CF
:1013000000F0ABF9030023707B68013B1A00FB6817
:10131000934205D20B4B180000F0CAF9031EE8D126
:10132000FB68002B06D03A68FB68D31800221A70BD
:10133000FB6800E000231800BD4605B090BDC04624
:1013400074030020BC02002080B584B000AF786038
:101350003960224B1B68002B02D101235B4238E02D
:101360007B684F2B0BDCC0461D4B180000F0A0F92A
:1013700003005022D21A7B689A42F5D302E002237E
:101380005B4226E00023FB600BE03A68FB68D31861
:101390001A78134B1100180000F02EF9FB68013386
:1013A000FB607B68FA689A42EFD30E4B1B680822F9
:1013B00013400DD10B4B1A680A4B08210A431A60DF
:1013C000074B180000F049F903001A00054B9A6218
:1013D00000231800BD4604B080BDC0467403002041
:1013E000180300200044004080B584B000AF78604E
:1013F00072B6C046454B00229A65444B9A6D434BEA
:101400005A65424B5A6D414B1A65414B00229A6511
:101410003F4B9A6D3E4B5A653D4B5A6D3C4B1A659E
:101420003C4B01221A603C4B00221A603B4BDA6AAB
:101430003A4B01210A43DA62394BFB607968F8685C
:1014400001F0D0FA0300FB60A023DB059A68A0231B
:10145000DB05802149050A439A60A023DB055A6811
:10146000A023DB052F490A405A60A023DB051B6837
:101470002D4A1A40A023DB05802189050A431A6002
:10148000A023DB055A6AA023DB058021C9040A4397
:101490005A62A023DB051B689B009A08A023DB058A
:1014A000802109060A431A60A023DB055A6AA0239B
:1014B000DB058021C9050A435A62184B9A6B174B0A
:1014C000802189020A439A63184B1A68174B6C21D2
:1014D0000A431A60154B00225A60144B00229A608E
:1014E000124BFA68DA60114B1A68104B01210A435B
:1014F0001A600F4B1A680E4B802149050A431A6087
:1015000062B6C046C046BD4604B080BDBC020020E5
:10151000180300207403002078030020001002400C
:101520000048E801FFBFFFFFFFFFFFCF004400407E
:1015300000E100E080B500AF084BDB69802213407A
:1015400001D000F025F8054BDB692022134001D0C3
:1015500000F006F8C046BD4680BDC04600440040CD
:1015600080B500AF074B5B6ADAB2074B1100180079
:1015700000F042F8031E02D0044B01221A60C0465C
:10158000BD4680BD00440040BC020020780300201E
:1015900080B500AF164B180000F08AF8031E08D083
:1015A000134B180000F059F803001A00114B9A620F
:1015B0001BE0104B1A680F4B08218A431A600D4B31
:1015C000DB694022134005D00A4B1A6A094B4021BF
:1015D0000A431A62074BDB698022134005D0054B92
:1015E0009A69044B10210A439A61C046BD4680BDEA
:1015F000180300200044004080B582B000AF78603E
:101600000A00FB1C1A707B681A6D7B685B6D9A423E
:1016100005D17B689B6D002B01D0012319E072B6C8
:10162000C0467B681B6D591C7A6811657A68F91C85
:101630000978D1547B689B6D5A1C7B689A657B68DE
:101640001B6D502B02D17B6800221A6562B6C04622
:1016500000231800BD4602B080BD80B584B000AF45
:1016600078607B689B6D002B01D100231CE072B673
:10167000C0467B685B6D591C7A6851650F22BA18A9
:101680007968CB5C13707B685B6D502B02D17B68F3
:1016900000225A657B689B6D5A1E7B689A6562B60C
:1016A000C0460F23FB181B781800BD4604B080BD50
:1016B00080B582B000AF78607B689B6D1800BD4636
:1016C00002B080BD80B582B000AF78600B4B1B6864
:1016D000002B09D101235B420BE07B685A1C7A6026
:1016E00019000120FFF730FE7B681B78002BF4D136
:1016F00000231800BD4602B080BDC0467403002020
:1017000080B582B000AF0200FB1D1A70FB1D1900EE
:101710000120FFF719FEC046BD4602B080BD80B56E
:1017200000AF044B1800FFF798FF03001800BD46F8
:1017300080BDC046BC020020B0B584B000AF786068
:1017400039601E4B1B68002B02D101235B4231E044
:101750000023FB600B23FB1800221A7017E0C04621
:10176000174B1800FFF7A4FF031EF9D00B257C19B7
:10177000134B1800FFF771FF03002370FB685A1C1E
:10178000FA601A007B689B187A1912781A703B6805
:10179000013BFA689A4204DA0B23FB181B780A2BE8
:1017A000DDD1FB68002B04DDFB687A68D3180022CA
:1017B0001A70FB681800BD4604B0B0BD7403002069
:1017C000BC02002080B500AF034B1800FFF770FF8C
:1017D00003001800BD4680BDBC02002090B583B058
:1017E00000AFFC1DFFF79BFF03002370FB1D1B7860
:1017F0001800FFF785FFFB1D1B781800BD4603B0DE
:1018000090BDB0B584B000AF78603960214B1B68E3
:10181000002B02D101235B4237E00023FB600B2346
:10182000FB1800221A701DE0C0461B4B1800FFF782
:101830003FFF031EF9D00B257C19174B1800FFF74B
:101840000CFF030023702C003B191B781800FFF7D6
:1018500057FFFB685A1CFA601A007B689B183A19FC
:1018600012781A703B68013BFA689A4204DA0B233B
:10187000FB181B780D2BD7D1FB68002B04DDFB6810
:101880007A68D31800221A70FB681800BD4604B0AD
:10189000B0BDC04674030020BC02002080B582B0F9
:1018A00000AF0200FB1D1A70FB1D1B781A001F23DE
:1018B000134001229A40034B1A60C046BD4602B055
:1018C00080BDC04600E100E080B500AF114B5A6B0F
:1018D000104B04210A435A630F4B104ADA6214205A
:1018E000FFF7DCFF0C4B1A680B4B10210A431A6000
:1018F000094B1A68084B01210A431A60064BDA6843
:10190000054B01210A43DA6062B6C046C046BD46B7
:1019100080BDC0460010024000080140FF7C00006E
:1019200080B582B000AF0200FB1D1A70FB1D1B7852
:101930001900104801F056F8030019000E4801F094
:1019400051F803005A1E0D4B5A600C4B00229A604E
:101950000A4B05221A60C046084B1A6880235B02B6
:101960001340F9D0054B00221A60C046BD4602B0B4
:1019700080BDC04640420F000048E80110E000E092
:1019800080B584B000AF78600023FB6015E00B23C6
:10199000FB1800221A7008E0FA20FFF7C1FF0B21A4
:1019A0007B181A787B1801321A700B23FB181B78EE
:1019B000032BF1D9FB680133FB60FA687B689A421C
:1019C000E5D3C046C046BD4604B080BD80B582B0F8
:1019D00000AF78607A68174B1100180004F09CFB88
:1019E000A023DB055A69A023DB0513490A405A618D
:1019F0000A20FFF7C5FF7B681800FFF763FE0F4B57
:101A00004F211800FFF798FEA023DB055A69A02399
:101A1000DB05802189010A435A610A20FFF7B0FFE4
:101A2000064A074B1100180004F076FBC046BD467D
:101A300002B080BDD88E0008FFDFFFFF80030020CA
:101A4000E48E000880B582B000AF786039603B68F2
:101A50007A680749074804F023FC064B1800FFF793
:101A600031FEC820FFF78CFFC046BD4602B080BDE6
:101A7000F48E00088003002080B500AFFFF7A2FEBF
:101A8000031E04DD034B4F211800FFF755FEC0462F
:101A9000BD4680BDD003002080B500AF034B1800C9
:101AA000FFF710FEC046BD4680BDC0468003002043
:101AB00080B500AFFFF786FE031E05DD044B4F2106
:101AC0001800FFF739FEC046C046BD4680BDC0467F
:101AD000D003002080B500AF134B1800FFF776FF4E
:101AE000124B1800FFF772FF114B1800FFF76EFF43
:101AF000104B1800FFF76AFF0F4B1800FFF766FF47
:101B00000E4B1800FFF762FF0D4B1800FFF75EFF4A
:101B10000C4B1800FFF75AFF0B4B1800FFF756FF4E
:101B2000C046BD4680BDC046FC8E00080C8F000834
:101B30001C8F0008288F0008348F0008408F000891
:101B40004C8F0008588F0008648F000890B587B04C
:101B500002AFF860B9607A60BC68FA680549064867
:101B60007B680093230004F09BFBC046BD4605B094
:101B700090BDC046708F00088003002090B585B0EE
:101B800000AF7860194B180004F0F8FB0300FB600D
:101B9000164B180003F000FB0300BB60BA68C823B3
:101BA0005B00D017D90F9A4248410300D9B2BB68F5
:101BB000F5225200DC0FD0179A4244412300DBB2D9
:101BC0000B40DBB2002B08D0B86801F07DFB031C92
:101BD000181C01F059FB030003E0786801F054FB86
:101BE00003001800BD4605B090BDC046D0030020DC
:101BF00080B500AF074B180004F0C0FB0300032BB7
:101C000005D9044A044B1100180004F085FAC046B7
:101C1000BD4680BDD0030020848F000880B500AF92
:101C2000A023DB055A69A023DB0502210A435A6180
:101C30002820FFF7EAFAA023DB055A69A023DB0579
:101C400002218A435A61C046BD4680BD80B582B03C
:101C500000AF0200FB1D1A70FB1D1B785BB2002B4E
:101C600008DAA023DB055A69A023DB0520210A43FB
:101C70005A6107E0A023DB055A69A023DB05202178
:101C80008A435A61FB1D1B784022134008D0A023D1
:101C9000DB055A69A023DB0510210A435A6107E0DE
:101CA000A023DB055A69A023DB0510218A435A6172
:101CB000FB1D1B782022134008D0A023DB055A69A6
:101CC000A023DB0508210A435A6107E0A023DB05B6
:101CD0005A69A023DB0508218A435A61FB1D1B7842
:101CE0001022134008D0A023DB055A69A023DB058E
:101CF00004210A435A6107E0A023DB055A69A023A7
:101D0000DB0504218A435A61FFF788FF2820FFF78B
:101D10007CFAFB1D1B780822134008D0A023DB05AA
:101D20005A69A023DB0520210A435A6107E0A0235A
:101D3000DB055A69A023DB0520218A435A61FB1D7C
:101D40001B780422134008D0A023DB055A69A02386
:101D5000DB0510210A435A6107E0A023DB055A691D
:101D6000A023DB0510218A435A61FB1D1B78022248
:101D7000134008D0A023DB055A69A023DB05082106
:101D80000A435A6107E0A023DB055A69A023DB055B
:101D900008218A435A61FB1D1B780122134008D099
:101DA000A023DB055A69A023DB0504210A435A61FD
:101DB00007E0A023DB055A69A023DB0504218A4341
:101DC0005A61FFF72BFFC046BD4602B080BD80B50B
:101DD00082B000AF0200FB1D1A70A023DB055A6918
:101DE000A023DB0501210A435A61FB1D1B78180063
:101DF000FFF72CFF0220FFF7F3F9C046BD4602B003
:101E000080BD80B582B000AF0200FB1D1A70A02318
:101E1000DB055A69A023DB0501218A435A61FB1DBA
:101E20001B781800FFF712FF0520FFF7D9F9C0460D
:101E3000BD4602B080BD80B500AFA023DB055A6966
:101E4000A023DB0502218A435A611420FFF7C8F959
:101E50003320FFF7D6FF3320FFF7D3FF3220FFF701
:101E6000D0FF2820FFF7CDFF0C20FFF7CAFF01208D
:101E7000FFF7C7FF1420FFF7B3F9C046BD4680BD8A
:101E800080B584B000AF786008001100FB1C021C14
:101E90001A70BB1C0A1C1A70FB1C1B78022B01D188
:101EA000C02300E080231800FFF7ABFF0520FFF7F9
:101EB00097F90023FB6009E0FB687A68D3181B7868
:101EC0001800FFF784FFFB680133FB60FB687A684A
:101ED000D3181B78002BEFD1BB1C1B78002B09D02B
:101EE00005E02020FFF773FFFB680133FB60FB6810
:101EF0000F2BF6DDC046BD4604B080BD80B500AFF7
:101F0000214B5A6B204B802189000A435A631F4B97
:101F10001A691E4BC02109060A431A611B4B1A6835
:101F20001A4B01210A431A60184B9A68174B01217A
:101F30000A439A60154BDA6880231B02134005D1CF
:101F4000C046124B1B6801221340FAD00F4B9B680E
:101F50000122134005D00D4B9A680C4B02210A4315
:101F60009A600A4B9A68094B802109060A439A60D5
:101F7000C046064B1A6880231B011340F9D0C046A7
:101F8000C046BD4680BDC04600100240002401404E
:101F900080B582B000AF7860164BDA68154B8021AF
:101FA00009020A43DA60134B7A689A62114B5A6944
:101FB000104B07210A435A617A6880239B029A4298
:101FC00006D10D4B1A680C4B8021C9030A431A60D5
:101FD000084B9A68074B04210A439A60C046054B98
:101FE0001B6804221340FAD0024B1B6C1800BD463C
:101FF00002B080BD002401400827014080B582B0B6
:1020000000AF0200FB1D1A70FB1D1B781A001F2376
:10201000134001229A40034B1A60C046BD4602B0ED
:1020200080BDC04600E100E080B500AF184B9A6B60
:10203000174B01210A439A638023DB05154ADA62B4
:102040000F20FFF7DBFF8023DB051A688023DB0509
:1020500010210A431A608023DB051A688023DB0500
:1020600080210A431A608023DB05DA688023DB05C0
:1020700001210A43DA608023DB051A688023DB052F
:1020800001210A431A6062B6C046C046BD4680BD03
:1020900000100240DF08000080B500AFA023DB0580
:1020A0005A69A023DB05802149004A405A61C04695
:1020B000BD4680BD80B584B000AF786039601B49F3
:1020C000786800F0D5FD031E03D0FE239B05FB605E
:1020D00020E01749786800F0C1FD031E03D080237B
:1020E000DB05FB6016E01349786800F0B7FD031EBE
:1020F00003D08123DB05FB600CE00F49786800F01A
:10210000ADFD031E03D08223DB05FB6002E08323C9
:10211000DB05FB60F968094800F0C8FD031CBB60E3
:10212000FB68181CBD4604B080BDC0460080D94382
:102130000080DE430080E3430080E84300005C460B
:1021400080B582B000AF78600021786800F080FD33
:10215000031E07D08023DB051B688023DB050022DC
:102160001A6007E08023DB051A688023DB05012164
:102170000A431A60C046BD4602B080BD80B500AFBC
:1021800000231800BD4680BDB0B584B000AF7860B4
:10219000FFF7F4FF0300FB60786802F055FE1F4A6A
:1021A0001F4B02F01DF802000B0010001900020086
:1021B0000B0001F0D7F802000B0010001900174ABD
:1021C000184B02F00DF802000B0014001D00786897
:1021D00002F03AFE02000B002000290002F000F895
:1021E00002000B000020104901F0F8FB02000B0078
:1021F00014001D00F86802F027FE02000B0020000A
:10220000290001F0EBFB02000B001000190002F0A6
:1022100093FE031C181CBD4604B0B0BD182D4454D9
:10222000FB211940FB2109400000F03F80B582B03E
:1022300000AF7860054B1B697A6813405A425341DE
:10224000DBB21800BD4602B080BDC046000400509D
:1022500080B582B000AF174B00221A70164B0122D6
:102260001A60164B180003F057FF154B180003F0C7
:10227000DFFF144B012201211800FFF701FE0023AC
:102280007B6007E0104A7B68D31820221A707B68B5
:1022900001337B607B68032BF4DD0B4B00221A714A
:1022A000094B012202211800FFF7EAFDC046BD4696
:1022B00002B080BD2004002024040020948F000878
:1022C000A08F0008B48F00082804002080B582B0D9
:1022D00000AF01235B427B608020FFF7A7FF031E56
:1022E0000FD14020FFF7A2FF031E0AD12020FFF7E5
:1022F0009DFF031E05D10820FFF798FF031E00D1A4
:102300008BE01E20FEF76CFF8020FFF78FFF031E7F
:1023100002D000237B601AE04020FFF787FF031EF6
:1023200002D001237B6012E02020FFF77FFF031E15
:1023300002D002237B600AE00820FFF777FF031E2C
:1023400002D003237B6002E001235B427B607B6859
:10235000002B10D1A023DB055A69A023DB05402107
:102360008A435A61A023DB055A69A023DB0580213B
:102370008A435A613AE07B68012B10D1A023DB0528
:102380005A69A023DB0540218A435A61A023DB055B
:102390005A69A023DB0580210A435A6126E07B6845
:1023A000022B10D1A023DB055A69A023DB054021B5
:1023B0000A435A61A023DB055A69A023DB0580216B
:1023C0008A435A6112E07B68032B0FD1A023DB05FF
:1023D0005A69A023DB0540210A435A61A023DB058B
:1023E0005A69A023DB0580210A435A61C046802038
:1023F000FFF71CFF031EFAD14020FFF717FF031E53
:10240000F5D12020FFF712FF031EF0D10820FFF7BF
:102410000DFF031EEBD17B6801E001235B42180036
:10242000BD4602B080BD80B582B000AFFFF74EFF61
:1024300003007B607B6801331AD00F4B1B781A00B6
:102440007B68934202D00D4B00221A600A4B1B7826
:102450001A000B4B2A219954094B01220221180022
:10246000FFF70EFD044B1B780133DAB2024B1A70F2
:10247000C046BD4602B080BD2004002024040020D8
:102480002804002080B500AFFFF7E2FE29E0184BDA
:102490001B78042B02D0FFF7C6FF22E0154B1B6808
:1024A000012B0DD1124B05221A70134B180003F0AB
:1024B000BFFE124B012201211800FFF7E1FC10E0E2
:1024C0000F4B180003F0B4FE0E4B0122012118003F
:1024D000FFF7D6FCFA239B001800FEF781FEFFF7FA
:1024E000B7FE034B1B78052BD1D1C046BD4680BD3E
:1024F0002004002024040020C48F0008D88F000886
:10250000E88F0008FC8F000880B582B000AF7860CB
:1025100039607B681B68181C02F0C6FC0022144B53
:1025200002F0CAF802000B001000190002F004FDCE
:10253000021C80231B065A407B681A603B681B689C
:10254000181C02F0B1FC00220A4B02F0B5F80200A0
:102550000B001000190002F0EFFC021C80231B0688
:102560005A403B681A60C046BD4602B080BDC046B6
:1025700000B0A04000F09F4080B584B000AF78600C
:1025800039600023FB60786802F08EFC2D4A2E4BE8
:1025900000F03EFB031E08D1786802F085FC2B4A50
:1025A0002B4B00F021FB031E47D00021786800F080
:1025B00073FB031E14D02749786800F03FFD031C0D
:1025C000181C02F071FC0022234B01F007FA0200F4
:1025D0000B001000190002F001FC0300FB6019E081
:1025E0000021786800F03AFB031E13D0194978687F
:1025F00000F024FD031C181C02F056FC0022174BAF
:1026000001F0ECF902000B001000190002F0E6FBEB
:102610000300FB603B68012B06D1FB68002B00DA4E
:1026200001335B10FB6008E03B68022B05D1FB68BF
:10263000002B00DA03339B10FB60FB681800BD46DB
:1026400004B080BD3433333333A35940CDCCCCCC2C
:10265000CC8C59C00000C8420006A04000F09F404A
:1026600080B584B000AF786039600023FB60786883
:1026700002F01AFC2D4A2E4B00F0CAFA031E08D1B4
:10268000786802F011FC2B4A2B4B00F0ADFA031EC8
:1026900047D00021786800F0FFFA031E14D02749C4
:1026A000786800F0CBFC031C181C02F0FDFB002234
:1026B000234B01F093F902000B001000190002F007
:1026C0008DFB0300FB6019E00021786800F0C6FA7A
:1026D000031E13D01949786800F0B0FC031C181CC5
:1026E00002F0E2FB0022174B01F078F902000B0028
:1026F0001000190002F072FB0300FB603B68012B25
:1027000006D1FB68002B00DA01335B10FB6008E0A8
:102710003B68022B05D1FB68002B00DA03339B10CA
:10272000FB60FB681800BD4604B080BDCDCCCCCCAE
:10273000CC7C58403433333333B35AC00000C842E2
:1027400000B0A040009C9E4080B582B000AF786091
:10275000FEE780B582B000AF786001235B421800CD
:10276000BD4602B080BD80B584B000AFF860B960EE
:102770007A60044B0C221A6001235B421800BD46AC
:1027800004B080BD4004002080B500AF034B0B2295
:102790001A6001235B421800BD4680BD4004002042
:1027A00080B582B000AF786039603B6880229201CA
:1027B0005A6000231800BD4602B080BD80B500AF4E
:1027C00001231800BD4680BD80B582B000AF78609F
:1027D0003960044B16221A6001235B421800BD4683
:1027E00002B080BD4004002080B582B000AF7860A8
:1027F0003960044B1F221A6001235B421800BD465A
:1028000002B080BD4004002080B584B000AFF86005
:10281000B9607A6000231800BD4604B080BD80B561
:1028200082B000AF786039603B68802292015A60C4
:1028300000231800BD4602B080BD80B582B000AF55
:10284000786001235B421800BD4602B080BD80B5B0
:1028500082B000AF7860044B02221A6001235B4211
:102860001800BD4602B080BD4004002080B582B093
:1028700000AF7860044B0A221A6001235B42180003
:10288000BD4602B080BDC0464004002080B582B085
:1028900000AF78607B68022B01D8012303E0044B72
:1028A00009221A6000231800BD4602B080BDC04650
:1028B0004004002080B586B000AF7860124B7B6189
:1028C000124B3B61124B1B68002B02D1104B7A69F3
:1028D0001A600F4B1B68FB600D4B1A687B68D3189E
:1028E0003A699A4205D20B4B0C221A6001235B42D3
:1028F00006E0074B1A687B68D218054B1A60FB6824
:102900001800BD4606B080BD5C0400200010002009
:102910003C0400204004002080B588B000AFF8607F
:10292000B9607A600023BB61FB68002B22D10023D1
:10293000FB611AE0FEF785FB03001A0017217B18E4
:102940001A70BB685A1CBA607A181278D2B21A7020
:10295000BB690133BB617B181B78DBB20A2B01D149
:10296000BB690EE0FB690133FB61FA697B689A423F
:10297000E0DB05E0054B09221A6001235B4200E021
:10298000BB691800BD4608B080BDC04640040020A9
:1029900080B586B000AFF860B9607A60FB68013B33
:1029A000012B11D800237B6109E0BB685A1CBA6077
:1029B0001B781800FEF736FB7B6901337B617A696F
:1029C0007B689A42F1DB05E0054B09221A6001237E
:1029D0005B4200E07B681800BD4606B080BDC04683
:1029E0004004002003460B437FD4002243088B425F
:1029F00074D303098B425FD3030A8B4244D3030B86
:102A00008B4228D3030C8B420DD3FF22090212BA4A
:102A1000030C8B4202D31212090265D0030B8B42C6
:102A200019D300E0090AC30B8B4201D3CB03C01AB0
:102A30005241830B8B4201D38B03C01A5241430B8B
:102A40008B4201D34B03C01A5241030B8B4201D37B
:102A50000B03C01A5241C30A8B4201D3CB02C01AE6
:102A60005241830A8B4201D38B02C01A5241430A5E
:102A70008B4201D34B02C01A5241030A8B4201D34D
:102A80000B02C01A5241CDD2C3098B4201D3CB01F4
:102A9000C01A524183098B4201D38B01C01A5241A3
:102AA00043098B4201D34B01C01A524103098B42A7
:102AB00001D30B01C01A5241C3088B4201D3CB0092
:102AC000C01A524183088B4201D38B00C01A524175
:102AD00043088B4201D34B00C01A5241411A00D225
:102AE00001465241104670475DE0CA0F00D049428E
:102AF000031000D34042534000229C4603098B42FE
:102B00002DD3030A8B4212D3FC22890112BA030A85
:102B10008B420CD3890192118B4208D38901921107
:102B20008B4204D389013AD0921100E08909C3098C
:102B30008B4201D3CB01C01A524183098B4201D38E
:102B40008B01C01A524143098B4201D34B01C01A79
:102B5000524103098B4201D30B01C01A5241C308F1
:102B60008B4201D3CB00C01A524183088B4201D360
:102B70008B00C01A5241D9D243088B4201D34B007B
:102B8000C01A5241411A00D20146634652415B10BD
:102B9000104601D34042002B00D54942704763469E
:102BA0005B1000D3404201B5002000F005F802BDE3
:102BB0000029F8D016E770477047C04684461000D9
:102BC00062468C461900634600E0C0461FB501F01E
:102BD000A3FA002801D40021C8421FBD10B501F09E
:102BE000F3F94042013010BD10B501F095FA00280C
:102BF00001DB002010BD012010BDC04610B501F062
:102C00008BFA002801DD002010BD012010BDC04658
:102C100010B501F01BFA002801DC002010BD0120D6
:102C200010BDC04610B501F011FA002801DA0020ED
:102C300010BD012010BDC046844608006146FFE774
:102C40001FB500F0B7F9002801D40021C8421FBD0C
:102C500010B500F043F94042013010BD10B500F04E
:102C6000A9F9002801DB002010BD012010BDC046DD
:102C700010B500F09FF9002801DD002010BD0120F3
:102C800010BDC04610B500F04FF9002801DC00204F
:102C900010BD012010BDC04610B500F045F9002858
:102CA00001DA002010BD012010BDC046F0B54F462E
:102CB0004646D6464502C0B547000C1C6D0A3F0E7D
:102CC000C60F002F00D170E0FF2F00D175E0EB00A0
:102CD0008025ED041D43002399469A467F3F6002FC
:102CE000430A984663001B0EE40F002B4ED0FF2BC7
:102CF00046D04246D0008022D204024390460022B1
:102D00007F3B3100FF1A4B466140C9B213430F2B82
:102D100000D9B5E06E489B00C3589F4600239846F3
:102D20002600454692465346022B00D189E0032BEC
:102D300000D19EE0012B18D03B007F33002B69DDD2
:102D40006A0704D00F222A40042A00D004352A0141
:102D500003D5604B1D403B008033FE2B00DD70E04F
:102D6000AD016D0AD8B202E00E0000200025C005BA
:102D70002843F6073043E0BCBA46B146A846F0BD4A
:102D80004346002B3FD10222FF3F03E04346002B86
:102D90002DD1012231004B466140C9B213430F2BA4
:102DA00034D84D489B00C3589F46002D13D10423AF
:102DB0009946033B00279A4691E7002D05D1082349
:102DC0009946063BFF279A4689E70C239946093B1B
:102DD000FF279A4683E7280002F0C0F97627431FB1
:102DE0009D4000237F4299469A463F1A77E7404626
:102DF00002F0B4F94246431F9A4076235B42904664
:102E00001B1A00227DE7FF2303227AE70E00FF2032
:102E10000025ACE70120C01A1B28A6DC9E372A003B
:102E2000BD40C2406B1E9D4115436B0704D00F236C
:102E30002B40042B00D004356B0144D50120002524
:102E400095E7FF20002592E780250026FF20ED036F
:102E50008DE7002398468020C003054209D04346F1
:102E6000034206D1454605436D022600FF206D0A48
:102E70007DE78020C00305436D02FF206D0A76E7E1
:102E800042466B015001834219D21B220025013FAB
:102E900001261C006D005B00002C01DB984201D86C
:102EA0001B1A3543013A002AF3D15A1E93411D43A0
:102EB0003B007F330E00002B00DD41E7AAE71A221A
:102EC00001251B1AE4E7AD0100206D0A4FE7C0465B
:102ED00010900008FFFFFFF75090000870B5420007
:102EE00045024E024C00C30F6D0A0120120E760AF5
:102EF000240EC90FFF2A06D0FF2C03D0A24201D115
:102F0000B54206D070BD002DFCD1FF2CFAD1002EA9
:102F1000F8D18B4206D00120002AF3D12800431EAD
:102F20009841EFE70020EDE770B5420045024E0200
:102F30004C00C30F6D0A120E760A240EC80FFF2A2A
:102F40001BD0FF2C0ED0002A1BD1002C01D1002E4B
:102F50001CD0002D0CD083421CD00221581E0840EA
:102F6000013870BD002E22D1002AF4D1002DF2D1FB
:102F70000028F6D101204042F3E7002D17D1FF2CA5
:102F8000F0D0002CE7D1002EE5D1E6E70020002D9F
:102F9000E7D0E2E7A24205DCEADBB54202D8E7D39C
:102FA0000020DEE74342584140000138D9E70220C3
:102FB0004042D6E770B5420045024E024C00C30FB6
:102FC0006D0A120E760A240EC80FFF2A0BD0FF2CB2
:102FD0000DD0002A1FD1002C16D1002E14D10020B4
:102FE000002D10D009E0002D0CD1FF2C13D1002EA4
:102FF00008D1002A08D0834212D00221581E08406E
:10300000013800E0022070BD002DF4D10028FAD173
:1030100001204042F7E7002CEDD1002EEBD1ECE788
:10302000A24205DCF2DBB54202D8EFD30020EAE78A
:103030004342584140000138E5E7C046F0B54F46ED
:103040004646D64644024500C0B5640A0F1C2D0E04
:10305000C60F002D00D18DE0FF2D00D192E000239E
:10306000802099469A46E400C00404437F3D7802DC
:10307000430A98467B001B0EFF0F002B00D170E027
:10308000FF2B00D186E04246D00080227F3BED1826
:103090000023D204024390469C4631004B467940BF
:1030A000681C0F2B1CD8764A9B00D3589F463900CA
:1030B0004446E2465346022B0FD0032B00D1D7E003
:1030C000012B37D100200024C0052043C907084345
:1030D000E0BCBA46B146A846F0BDFF200024F3E7A5
:1030E000260C2404220C44462404240C43462700C6
:1030F0001B0C574374435A435E4312193B0C9B18F5
:103100009C4203D980225202944666443F041A042A
:103110003F0CD2199401671EBC411B0C920E9B19E7
:1031200014439B011C431B0100D49BE00123620854
:103130001C40144302007F32002A64DD630704D080
:103140000F232340042B00D00434230103D50200B5
:103150004C4B80321C40FE2ABFDCA401640AD0B272
:10316000B2E74346002B3DD14A4601331A4391460C
:103170009C4692E7002C29D104239946033B002565
:103180009A4674E7002C1BD108239946063BFF257D
:103190009A466CE74346FF35002B0BD102234A4683
:1031A0001A4391469C4678E753463100022B00D0E3
:1031B00083E792E703234A461A4391469C466CE70D
:1031C0000C239946093BFF259A4650E7200001F061
:1031D000C5FF7625431F9C4000236D4299469A46C1
:1031E0002D1A44E7404601F0B9FF4246431F9A407A
:1031F00000232D1A90469C46763D4EE78024002100
:10320000FF20E40360E701239B1A1B2B00DD59E735
:1032100022009E30DA4084401300621E94411C4319
:10322000630704D00F232340042B00D00434630130
:103230001AD50120002447E78020C003044209D0AA
:103240004346034206D14446044364023900FF204A
:10325000640A39E78020C003044364023100FF2080
:10326000640A31E7280065E7A4010020640A2BE71F
:103270008020C00304436402FF20640A24E7C046A0
:1032800090900008FFFFFFF741024200C30F490A78
:103290000020120E7E2A03DD9D2A02DD094A9818BD
:1032A0007047802000040143952A07DC9620821A8B
:1032B000D1404842002BF3D10800F1E7963A914003
:1032C000F7E7C046FFFFFF7FF8B5002813D0C3170C
:1032D000C6185E40C40F300001F040FF9E23050079
:1032E0001B1A962B0FDC082801DD083DAE40760244
:1032F000760AD8B202E0002400200026C005304340
:10330000E4072043F8BD992B0CDD05223100121A89
:10331000D1400A00010030001B318840411E884125
:1033200002431600052D12DC31000D4F39407207A3
:1033300009D00F203040042805D004314A0102D5BD
:103340009F2339405B1B89014E0AD8B2D6E76A1F1A
:1033500096403100024F39407207F4D0E9E7C04689
:10336000FFFFFFFBF0B54F464646D6460D00040072
:10337000C0B51F0011002803620F400A10437A00F5
:10338000520DE3003C039146640AFA0F4F0F6E00A2
:1033900027439246B846760DED0FC900954200D1FD
:1033A00099E04C46341BA446002C00DC7CE04A46E5
:1033B000002A00D1B8E0C54A964200D11CE1802223
:1033C0003C0012041443A0466246382A00DD61E145
:1033D0001F2A00DDCCE164462022121B44469440A3
:1033E0000F00A14664469140E7404C464A1E914179
:1033F0003C43424621436446E240801A5C1AA342A1
:103400009B415F42C71B3B0200D4D0E07F027F0A92
:10341000002F00D1FFE0380001F0A0FE01000839C4
:10342000202322005B1A8F40DA408C401743B142C0
:1034300000DAFFE0891B4B1C1F2B00DDA8E02022D7
:103440003900D21A200094409140D840621E944125
:10345000DF40002601430C43630709D00F232340BC
:10346000042B05D0231DA342A44164423F191C0034
:103470003B0200D49EE0954B01369E4200D1B7E05E
:10348000934AE40817407B0771057F0223433F0BF3
:103490004A0D12053A43ED072A4318001100E0BC1B
:1034A000BA46B146A846F0BD002C4BD04C46A41BF2
:1034B000A446002E00D023E104001C4300D1AFE15C
:1034C0006246541E012A00D115E2804DAC4500D160
:1034D000C8E1A4461BE14A46B21A9446002A00DC21
:1034E000ACE04A46002A43D0784A964200D1AFE188
:1034F00080223C0012041443A0466246382A67DC4E
:103500001F2A00DC5FE14746203AD7406246202A66
:1035100005D064464022121B4446944021434A1E73
:1035200091410C003C4357E03A000A4300D105E1C9
:103530002200013A012C00D182E1644CA4455BD009
:10354000944641E7634C771C274200D0C4E0040056
:103550001C43002E00D069E1002C00D1BFE144469D
:103560000C4300D0D0E14207DB081343C00829E038
:103570003A000A4300D170E162466446013A012CE8
:1035800000D1E0E0514CA44500D161E19446B4E79C
:103590003A001F39CA401100202B03D04022D31A11
:1035A0009F403C43631E9C41002700260C43630759
:1035B00000D053E7B446E4087B072343F808434AA6
:1035C00094451DD06246070352053F0B520D60E73C
:1035D00044460C43621E9441E4189C429B415F4266
:1035E0003F183B02E3D5394B01369E4200D0B5E08F
:1035F0003200002700234CE74207DB081343C008D2
:103600001A00024300D1E1E180273F0307433F0353
:103610002E4A3F0B3DE7200001F0A0FD01001831CC
:103620001F2900DCFCE60838844027000024B14252
:1036300000DBFFE6264A761A17400DE7002A2FD056
:103640004A46921B9446002E00D1ADE01F4A914598
:1036500000D10FE18022120410436246382A00DDB7
:103660000FE11F2A00DD80E1644620221E00121BAC
:103670006746040093409440FE405A1E9341F84030
:1036800034431C43804464188C42BF417F424E4601
:103690004744A6E742460A4311004A1E9141ADE65F
:1036A0000C4C721C224200D0A1E002001A43002EF2
:1036B00000D0FAE0002A00D145E13A000A4300D0E8
:1036C00046E14207DB081343C0087BE7FF07000021
:1036D000FFFF7FFFFE07000047465C1AC21BA342A4
:1036E000BF417F42B94617004A46BF1A3A0200D589
:1036F0008DE023003B4300D08AE60020002561E7EF
:10370000B44CA14500D1ADE080242404204364469C
:10371000382C3DDC62461F2C00DDB7E020251E0062
:103720002D1B0400AB40AC40D640D04042465D1E4D
:10373000AB413443121A904623432CE04207DB0886
:103740001343C0083BE75C189C429B4140445B42EA
:10375000C71801263B0200D429E702269E4A6308C7
:103760001740012214401C43FB071C437F0873E6EB
:103770004446203AD4406246202A05D0674640227B
:10378000D21B4746974039434A1E9141214335E6B3
:103790000343581E8341CC1AA142BF4143467F4296
:1037A00055464E46DF1B2EE602001A4300D1BDE00F
:1037B00062466446013A012C00D1E5E0854CA445FF
:1037C00058D0944649E764462022121B4446944050
:1037D0000F00A14664469140E7404C464A1E914185
:1037E0003C4342460C436146CA408018F4E6794C9B
:1037F000A24200D1FDE6591899429B4140445F42E4
:10380000C719FC07490816000C437F08CFE6CC1AFD
:10381000A142BF4143467F42181A5546C71BF7E5F0
:10382000C9087B0755460B43F808C8E6002C00D0B2
:1038300081E043460B4315D1802000250003E3E6D9
:103840005C1AA3429B41C71B5B420126FF1ADAE5C3
:103850004207DB081343C008D2E64207DB081343E4
:10386000C008ACE643464246C9085B0755460B43D1
:10387000D008C5E6434642465B07C9080B43D0085B
:10388000BEE603431C00631E9C41FCE60200203C94
:10389000E24014006246202A03D04025AD1AA84019
:1038A0000343581E8341234375E7002AE2D03A00C0
:1038B0000A43CDD04207DB0813438022C00812031D
:1038C000104206D0FC08144203D12000CB087A072E
:1038D00013435A0FDB005207DB08134390E64346BD
:1038E0000B4300D109E743464246C9085B075546EA
:1038F0000B43D00866E6CC1AA14289413F1A4942DF
:10390000554601267F1A7EE542465C1A871AA34275
:1039100092415242BF1A3A023DD5CC1AA142894186
:10392000434649421F1A55467F1A95E57B07C90849
:103930000B43F80843E64446DB080C4330D142070A
:103940001343C0085CE67B07C9080B43F80839E657
:103950005C189C429B4140445B42C7183B0200D428
:1039600025E61D4B01261F4021E60400203AD440E5
:103970006246202A04D040226646921B90400343B0
:103980005A1E93411C437EE65C188C428941404498
:1039900049424718DDE623003B4300D1ADE606E689
:1039A000440723438024C0082403204208D0424611
:1039B000D608264204D155463000CB0851070B43A8
:1039C0005A0FDB00DB085207134319E60023014AB4
:1039D0001F005EE5FF070000FFFF7FFFF0B55746C1
:1039E0004E464546DE46E0B5814605000C034800DC
:1039F00092461F0085B0240B400DCE0F002800D149
:103A000056E1D44B984200D172E16B0FE4001C43A5
:103A100080231B0423439846CF4BED009B46002395
:103A20009946834400933C037B005046240B5B0D76
:103A3000FF0F002B00D11FE1C64A934200D162E183
:103A4000C549420F8C46E400594614438022634422
:103A50001204CB1A14439B46C200002033007B4063
:103A60009A464B460F2B27D8BC499B00CB589F4604
:103A7000B246009B022B16D0032B00D18EE2012B05
:103A800000D0D9E000230024002552461B05234323
:103A9000D20713432800190005B0F0BCBB46B2465C
:103AA000A946A046F0BD00240025AA4BEDE7BA4682
:103AB000A04615000090DCE7444500D2C7E100D1E4
:103AC000C2E101235B429C462E0040460025E344B0
:103AD0002302140E1C431B0C994623041F0C1202D4
:103AE00049460092019701F035FB02007A430B042E
:103AF000310C804619438A4207D901235B429C4618
:103B00000919E0448C4200D807E2881A494601F0BE
:103B100021FB09048C4631046646019A090C424394
:103B2000030031438A4204D90919013B8C4200D871
:103B3000EDE1881A424612041A4390464146009B22
:103B40000E041B0C1F000293009B360C1B04190C67
:103B50000B007343120C7E43039151437A431F0CB5
:103B6000BC4676186644B14203D9802149028C468E
:103B70006244310C8A1831041E04360C8E199042AE
:103B800002D312D1B54210D24346591E009B9C4627
:103B900065441F009D429B415B421B19C018844233
:103BA00000D2A0E100D19BE18846AE1BB542AD41F9
:103BB000801A6D42401B844200D1D5E1494601F094
:103BC000C9FA019A0B044243310C050019438A4299
:103BD00000D96CE1881A494601F0BCFA019A360412
:103BE00042430904360C03000E43B24200D953E1AC
:103BF0000398B61A02002D041D43029F2B041B0CD0
:103C00005A437B439C46290C4843130C8444634429
:103C10007943984203D98020400284466144180CBD
:103C200012041B04120C41189B188E4200D2FFE0B4
:103C300000D1FAE001231D43494A5A44002A00DC1E
:103C4000AAE06B0700D03DE1ED084346DB0106D555
:103C50004246444B1A4090468022D2005A44424B7E
:103C60009A4200DD1FE743465B071D43434652056A
:103C70005C02240B530D08E75246224300D17BE03F
:103C8000002C00D1FAE0200001F068FA02000B3AA3
:103C90001D2301009B1A52460839DA408C40144318
:103CA00052468A40314B58449B4683440020D5E617
:103CB0004B462343984644D0002C00D1CEE0200050
:103CC00001F04CFA010002000B391D235B1A494632
:103CD0001000D940083884400B004D4623439846D5
:103CE00085402348831A9B460023994600939AE611
:103CF0004B46234398461DD108239946063B002591
:103D0000834600938FE65246224309D10223494657
:103D10001943184B89469C4600240220E3449DE643
:103D200003234A461A43134B91469C4652460320AE
:103D3000E34493E60C239946093BA046834600934F
:103D400071E60423994600239B4601330025009326
:103D500069E6C046FF07000001FCFFFFD0900008A5
:103D6000FF030000FFFFFFFEFE070000F30300005B
:103D70000DFCFFFF01F8FFFF494601231943894667
:103D8000002401206AE6002380249A4600258A4BFD
:103D900024037AE601256D4201239B1A382B00DDAE
:103DA00070E61F2B00DCBFE01F2149428A1A414602
:103DB000D1400A00202B04D04146804B5B449940FF
:103DC0000D436B1E9D4107232A431D00002415400F
:103DD000134200D1D4E00F2100231140042900D167
:103DE000CBE0111D9142924152429B180A001902E8
:103DF00000D4C2E001230024002546E6802341468A
:103E00001B03194208D01C4206D11C432403BA46A6
:103E10001500694B240B38E68024434624031C43D9
:103E20002403B246644B240B2FE6002B00D103E79A
:103E3000A619681EA64200D28DE08E4200D2A3E0F1
:103E400000D1B3E00500F5E6AA4200D939E64346C1
:103E5000DE0758086B081E43ED0739E6484601F0B7
:103E60007DF901000200153120321C2900DC2CE70D
